 lcdcbacklight

 Timestamp is 4da2a52d (Mon Apr 11 18:52:29 2011)

 Preferred load address is 10000000

 Start         Length     Name                   Class
 0001:00000000 00000004H .CRT$XCA                CODE
 0001:00000004 00000004H .CRT$XCZ                CODE
 0001:00000008 00000004H .CRT$XIA                CODE
 0001:0000000c 00000004H .CRT$XIZ                CODE
 0001:00000010 00000004H .CRT$XPA                CODE
 0001:00000014 00000004H .CRT$XPZ                CODE
 0001:00000018 00000004H .CRT$XTA                CODE
 0001:0000001c 00000004H .CRT$XTZ                CODE
 0001:00000020 000012bcH .rdata                  CODE
 0001:000012dc 0000002aH .rdata$debug            CODE
 0001:00001308 00002e2cH .text                   CODE
 0001:00004134 00000008H .xdata                  CODE
 0001:0000413c 0000003cH .idata$2                CODE
 0001:00004178 00000014H .idata$3                CODE
 0001:0000418c 000000b4H .idata$4                CODE
 0001:00004240 00000078H .idata$6                CODE
 0001:000042c0 00000105H .edata                  CODE
 0002:00000000 000000b4H .idata$5                DATA
 0002:000000b8 000004e4H .data                   DATA
 0002:0000059c 0000009cH .bss                    DATA
 0003:00000000 00000130H .pdata                  DATA

  Address         Publics by Value              Rva+Base       Lib:Object

 0000:00000000       ___safe_se_handler_count   00000000     <absolute>
 0000:00000000       ___safe_se_handler_table   00000000     <absolute>
 0001:00000000       __xc_a                     10001000     corelib0:crt0init.obj
 0001:00000004       __xc_z                     10001004     corelib0:crt0init.obj
 0001:00000008       __xi_a                     10001008     corelib0:crt0init.obj
 0001:0000000c       __xi_z                     1000100c     corelib0:crt0init.obj
 0001:00000010       __xp_a                     10001010     corelib0:crt0init.obj
 0001:00000014       __xp_z                     10001014     corelib0:crt0init.obj
 0001:00000018       __xt_a                     10001018     corelib0:crt0init.obj
 0001:0000001c       __xt_z                     1000101c     corelib0:crt0init.obj
 0001:0000003c       ??_C@_19OBGHODPD@?$AAM?$AAo?$AAd?$AAe?$AA?$AA@ 1000103c     bspbacklight.obj
 0001:00000048       ??_C@_1CK@ENPFCICM@?$AAD?$AAr?$AAi?$AAv?$AAe?$AAr?$AAs?$AA?2?$AAD?$AAi?$AAs?$AAp?$AAl?$AAa?$AAy?$AA?2?$AAL?$AAC?$AAD?$AAC?$AA?$AA@ 10001048     bspbacklight.obj
 0001:00000074       ??_C@_1CM@JBPFNDBJ@?$AAD?$AAr?$AAi?$AAv?$AAe?$AAr?$AAs?$AA?2?$AAB?$AAu?$AAi?$AAl?$AAt?$AAI?$AAn?$AA?2?$AAL?$AAC?$AAD?$AAA?$AAD?$AA?$AA@ 10001074     bspbacklight.obj
 0001:000000a0       ??_C@_1CA@CPJPALBJ@?$AAB?$AAK?$AAL?$AA_?$AAI?$AAN?$AAI?$AAT?$AA?$CI?$AA?$CJ?$AA?5?$AA?9?$AA?$CB?$AA?$AN?$AA?6?$AA?$AA@ 100010a0     backlight_common_topaz_v1:backlight.obj
 0001:000000c0       ??_C@_1HE@OFKIAIPG@?$AAB?$AAK?$AAL?$AA_?$AAI?$AAn?$AAi?$AAt?$AA?3?$AA?5?$AAF?$AAa?$AAi?$AAl?$AAe?$AAd?$AA?5?$AAt?$AAo?$AA?5?$AAc?$AAr?$AAe?$AAa?$AAt?$AAe?$AA?5?$AAB?$AAL?$AAD?$AA?5?$AAI@ 100010c0     backlight_common_topaz_v1:backlight.obj
 0001:00000134       ??_C@_1DC@NCJLNBML@?$AAB?$AAK?$AAL?$AA_?$AAI?$AAn?$AAi?$AAt?$AA?3?$AA?5?$AAC?$AAr?$AAe?$AAa?$AAt?$AAe?$AAT?$AAh?$AAr?$AAe?$AAa?$AAd?$AA?$AN?$AA?6?$AA?$AA@ 10001134     backlight_common_topaz_v1:backlight.obj
 0001:00000168       ??_C@_1EE@BMCHIEHD@?$AAC?$AAr?$AAe?$AAa?$AAt?$AAe?$AA?5?$AAB?$AAK?$AAL?$AA_?$AAC?$AAH?$AAA?$AAN?$AAG?$AAE?$AA?5?$AAe?$AAv?$AAe?$AAn?$AAt?$AA?5?$AAf?$AAa?$AAi?$AAl?$AAe?$AAd?$AA?$CB?$AA?$AN@ 10001168     backlight_common_topaz_v1:backlight.obj
 0001:000001ac       ??_C@_1DA@IKPIDNLP@?$AAB?$AAK?$AAL?$AAC?$AAh?$AAa?$AAn?$AAg?$AAe?$AAI?$AAn?$AAC?$AAo?$AAn?$AAt?$AAr?$AAo?$AAl?$AAP?$AAa?$AAn?$AAe?$AAl?$AA?$AA@ 100011ac     backlight_common_topaz_v1:backlight.obj
 0001:000001e0       ??_C@_1FC@OPKONBOL@?$AAG?$AAe?$AAt?$AA?5?$AAB?$AAa?$AAc?$AAk?$AAL?$AAi?$AAg?$AAh?$AAt?$AAL?$AAe?$AAv?$AAe?$AAl?$AAC?$AAh?$AAa?$AAn?$AAg?$AAe?$AAE?$AAv?$AAe?$AAn?$AAt?$AA?5?$AAf?$AAa@ 100011e0     backlight_common_topaz_v1:backlight.obj
 0001:00000234       ??_C@_1DE@PFEDGFDL@?$AAB?$AAa?$AAc?$AAk?$AAL?$AAi?$AAg?$AAh?$AAt?$AAL?$AAe?$AAv?$AAe?$AAl?$AAC?$AAh?$AAa?$AAn?$AAg?$AAe?$AAE?$AAv?$AAe?$AAn?$AAt?$AA?$AA@ 10001234     backlight_common_topaz_v1:backlight.obj
 0001:00000268       ??_C@_1DM@GAJKEPGB@?$AAC?$AAr?$AAe?$AAa?$AAt?$AAe?$AA?5?$AAd?$AAu?$AAm?$AAm?$AAy?$AA?5?$AAe?$AAv?$AAe?$AAn?$AAt?$AA?5?$AAf?$AAa?$AAi?$AAl?$AAe?$AAd?$AA?$CB?$AA?$CB?$AA?$AN?$AA?6?$AA?$AA@ 10001268     backlight_common_topaz_v1:backlight.obj
 0001:000002a8       ??_C@_1EK@HLKMLPAD@?$AAG?$AAe?$AAt?$AA?5?$AAU?$AAs?$AAe?$AAr?$AA?5?$AAI?$AAn?$AAa?$AAc?$AAt?$AAi?$AAv?$AAi?$AAt?$AAy?$AA?5?$AAE?$AAv?$AAe?$AAn?$AAt?$AA?5?$AAf?$AAa?$AAi?$AAl?$AAe?$AAd@ 100012a8     backlight_common_topaz_v1:backlight.obj
 0001:000002f8       ??_C@_1EG@KHBDFHDI@?$AAP?$AAo?$AAw?$AAe?$AAr?$AAM?$AAa?$AAn?$AAa?$AAg?$AAe?$AAr?$AA?1?$AAU?$AAs?$AAe?$AAr?$AAA?$AAc?$AAt?$AAi?$AAv?$AAi?$AAt?$AAy?$AA_?$AAI?$AAn?$AAa?$AAc?$AAt?$AAi@ 100012f8     backlight_common_topaz_v1:backlight.obj
 0001:00000340       ??_C@_1EG@FKHCPIKF@?$AAG?$AAe?$AAt?$AA?5?$AAU?$AAs?$AAe?$AAr?$AA?5?$AAA?$AAc?$AAt?$AAi?$AAv?$AAi?$AAt?$AAy?$AA?5?$AAE?$AAv?$AAe?$AAn?$AAt?$AA?5?$AAf?$AAa?$AAi?$AAl?$AAe?$AAd?$AA?$CB?$AA?$CB@ 10001340     backlight_common_topaz_v1:backlight.obj
 0001:00000388       ??_C@_1EC@PPGKBJLE@?$AAP?$AAo?$AAw?$AAe?$AAr?$AAM?$AAa?$AAn?$AAa?$AAg?$AAe?$AAr?$AA?1?$AAU?$AAs?$AAe?$AAr?$AAA?$AAc?$AAt?$AAi?$AAv?$AAi?$AAt?$AAy?$AA_?$AAA?$AAc?$AAt?$AAi?$AAv?$AAe@ 10001388     backlight_common_topaz_v1:backlight.obj
 0001:000003d0       ??_C@_1EM@KJMLPDDB@?$AAR?$AAe?$AAq?$AAu?$AAe?$AAs?$AAt?$AA?5?$AAP?$AAo?$AAw?$AAe?$AAr?$AA?5?$AAN?$AAo?$AAt?$AAi?$AAf?$AAi?$AAc?$AAa?$AAt?$AAi?$AAo?$AAn?$AA?5?$AAf?$AAa?$AAi?$AAl?$AA?$CB@ 100013d0     backlight_common_topaz_v1:backlight.obj
 0001:0000041c       ??_C@_1DA@KADEIHFA@?$AAC?$AAr?$AAe?$AAa?$AAt?$AAe?$AA?5?$AAM?$AAs?$AAg?$AAQ?$AAu?$AAe?$AAu?$AAe?$AA?5?$AAf?$AAa?$AAi?$AAl?$AA?$CB?$AA?$CB?$AA?6?$AA?$AA@ 1000141c     backlight_common_topaz_v1:backlight.obj
 0001:00000450       ??_C@_1EI@GLMEKADC@?$AAG?$AAe?$AAt?$AA?5?$AAB?$AAa?$AAc?$AAk?$AAL?$AAi?$AAg?$AAh?$AAt?$AAC?$AAh?$AAa?$AAn?$AAg?$AAe?$AAE?$AAv?$AAe?$AAn?$AAt?$AA?5?$AAf?$AAa?$AAi?$AAl?$AAe?$AAd?$AA?$CB@ 10001450     backlight_common_topaz_v1:backlight.obj
 0001:00000498       ??_C@_1CK@NJCEAPDJ@?$AAB?$AAa?$AAc?$AAk?$AAL?$AAi?$AAg?$AAh?$AAt?$AAC?$AAh?$AAa?$AAn?$AAg?$AAe?$AAE?$AAv?$AAe?$AAn?$AAt?$AA?$AA@ 10001498     backlight_common_topaz_v1:backlight.obj
 0001:000004c4       ??_C@_1CM@GOAMMABD@?$AAd?$AAe?$AAv?$AAi?$AAc?$AAe?$AA?5?$AAn?$AAa?$AAm?$AAe?$AA?5?$AAi?$AAs?$AA?5?$AA?8?$AA?$CF?$AAs?$AA?8?$AA?$AN?$AA?6?$AA?$AA@ 100014c4     backlight_common_topaz_v1:backlight.obj
 0001:000004f0       ??_C@_1GE@CKDEJCGE@?$AAB?$AAK?$AAL?$AA_?$AAI?$AAn?$AAi?$AAt?$AA?3?$AA?5?$AAR?$AAe?$AAg?$AAQ?$AAu?$AAe?$AAr?$AAy?$AAV?$AAa?$AAl?$AAu?$AAe?$AAE?$AAx?$AA?$CI?$AA?8?$AA?$CF?$AAs?$AA?8?$AA?0?$AA?5@ 100014f0     backlight_common_topaz_v1:backlight.obj
 0001:00000554       ??_C@_19DINFBLAK@?$AAN?$AAa?$AAm?$AAe?$AA?$AA@ 10001554     backlight_common_topaz_v1:backlight.obj
 0001:00000560       ??_C@_1FE@DEAJHAEE@?$AAB?$AAK?$AAL?$AA_?$AAI?$AAn?$AAi?$AAt?$AA?3?$AA?5?$AAO?$AAp?$AAe?$AAn?$AAD?$AAe?$AAv?$AAi?$AAc?$AAe?$AAK?$AAe?$AAy?$AA?$CI?$AA?8?$AA?$CF?$AAs?$AA?8?$AA?$CJ?$AA?5?$AAf?$AAa@ 10001560     backlight_common_topaz_v1:backlight.obj
 0001:000005b4       ??_C@_1CA@CCIBHLFO@?$AAB?$AAK?$AAL?$AA_?$AAI?$AAN?$AAI?$AAT?$AA?$CI?$AA?$CJ?$AA?5?$AA?$CL?$AA?$CB?$AA?$AN?$AA?6?$AA?$AA@ 100015b4     backlight_common_topaz_v1:backlight.obj
 0001:000005d4       ??_C@_1BM@HPLBBPGP@?$AA?9?$AAB?$AAK?$AAL?$AA_?$AAD?$AAe?$AAi?$AAn?$AAi?$AAt?$AA?$AN?$AA?6?$AA?$AA@ 100015d4     backlight_common_topaz_v1:backlight.obj
 0001:000005f0       ??_C@_1EA@GOCLCMDH@?$AA?$CL?$AAB?$AAK?$AAL?$AA_?$AAD?$AAe?$AAi?$AAn?$AAi?$AAt?$AA?3?$AA?5?$AAd?$AAw?$AAC?$AAo?$AAn?$AAt?$AAe?$AAx?$AAt?$AA?5?$AA?$DN?$AA?5?$AA0?$AAx?$AA?$CF?$AAx?$AA?$AN?$AA?6?$AA?$AA@ 100015f0     backlight_common_topaz_v1:backlight.obj
 0001:00000630       ??_C@_1BO@BCGBANIP@?$AAW?$AAA?$AAI?$AAT?$AA_?$AAF?$AAA?$AAI?$AAL?$AAE?$AAD?$AA?$CB?$AA?$AN?$AA?6?$AA?$AA@ 10001630     backlight_common_topaz_v1:backlight.obj
 0001:00000650       ??_C@_1DM@OACLIHDI@?$AAn?$AAe?$AAw?$AA?5?$AAb?$AAa?$AAc?$AAk?$AAl?$AAi?$AAg?$AAh?$AAt?$AA?5?$AAa?$AAc?$AA?5?$AAl?$AAe?$AAv?$AAe?$AAl?$AA?5?$AA?$DN?$AA?5?$AA?$CF?$AAd?$AA?$AN?$AA?6?$AA?$AA@ 10001650     backlight_common_topaz_v1:backlight.obj
 0001:00000690       ??_C@_1EA@IMNHGGLN@?$AAn?$AAe?$AAw?$AA?5?$AAb?$AAa?$AAc?$AAk?$AAl?$AAi?$AAg?$AAh?$AAt?$AA?5?$AAb?$AAa?$AAt?$AAt?$AA?5?$AAl?$AAe?$AAv?$AAe?$AAl?$AA?5?$AA?$DN?$AA?5?$AA?$CF?$AAd?$AA?$AN?$AA?6?$AA?$AA@ 10001690     backlight_common_topaz_v1:backlight.obj
 0001:000006d0       ??_C@_1DE@HJBKBBNP@?$AAb?$AAa?$AAc?$AAk?$AAl?$AAi?$AAg?$AAh?$AAt?$AA?5?$AAa?$AAc?$AA?5?$AAl?$AAe?$AAv?$AAe?$AAl?$AA?5?$AA?$DN?$AA?5?$AA?$CF?$AAd?$AA?$AN?$AA?6?$AA?$AA@ 100016d0     backlight_common_topaz_v1:backlight.obj
 0001:00000704       ??_C@_1DI@HBGPPHCM@?$AAb?$AAa?$AAc?$AAk?$AAl?$AAi?$AAg?$AAh?$AAt?$AA?5?$AAb?$AAa?$AAt?$AAt?$AA?5?$AAl?$AAe?$AAv?$AAe?$AAl?$AA?5?$AA?$DN?$AA?5?$AA?$CF?$AAd?$AA?$AN?$AA?6?$AA?$AA@ 10001704     backlight_common_topaz_v1:backlight.obj
 0001:00000740       ??_C@_1EM@CKOKHOMN@?$AA?$CF?$AAs?$AA?3?$AA?5?$AAD?$AAe?$AAv?$AAi?$AAc?$AAe?$AAP?$AAo?$AAw?$AAe?$AAr?$AAN?$AAo?$AAt?$AAi?$AAf?$AAy?$AA?$CI?$AAD?$AA0?$AA?$CJ?$AA?5?$AAf?$AAa?$AAi?$AAl?$AAe?$AAd@ 10001740     backlight_common_topaz_v1:backlight.obj
 0001:00000790       ??_C@_1EM@NLGJPCON@?$AA?$CF?$AAs?$AA?3?$AA?5?$AAD?$AAe?$AAv?$AAi?$AAc?$AAe?$AAP?$AAo?$AAw?$AAe?$AAr?$AAN?$AAo?$AAt?$AAi?$AAf?$AAy?$AA?$CI?$AAD?$AA4?$AA?$CJ?$AA?5?$AAf?$AAa?$AAi?$AAl?$AAe?$AAd@ 10001790     backlight_common_topaz_v1:backlight.obj
 0001:000007dc       ??_C@_1DA@PJJNJDEO@?$AAR?$AAe?$AAa?$AAd?$AAM?$AAs?$AAg?$AAQ?$AAu?$AAe?$AAu?$AAe?$AA?3?$AA?5?$AAE?$AAR?$AAR?$AAO?$AAR?$AA?3?$AA?$CF?$AAd?$AA?6?$AA?$AA@ 100017dc     backlight_common_topaz_v1:backlight.obj
 0001:0000080c       ??_C@_1CK@JHECJOND@?$AAb?$AAA?$AAC?$AAO?$AAn?$AAl?$AAi?$AAn?$AAe?$AA?5?$AA?$DN?$AA?5?$AAF?$AAA?$AAL?$AAS?$AAE?$AA?$DL?$AA?$AN?$AA?6?$AA?$AA@ 1000180c     backlight_common_topaz_v1:backlight.obj
 0001:00000838       ??_C@_1CI@DENCAJKG@?$AAb?$AAA?$AAC?$AAO?$AAn?$AAl?$AAi?$AAn?$AAe?$AA?5?$AA?$DN?$AA?5?$AAT?$AAR?$AAU?$AAE?$AA?$DL?$AA?$AN?$AA?6?$AA?$AA@ 10001838     backlight_common_topaz_v1:backlight.obj
 0001:00000860       ??_C@_1DG@BHBJAMBN@?$AAL?$AAi?$AAn?$AAe?$AA?5?$AAs?$AAt?$AAa?$AAt?$AAu?$AAs?$AA?5?$AAi?$AAs?$AA?5?$AA?$CF?$AAs?$AA?5?$AA?$CI?$AA0?$AAx?$AA?$CF?$AAx?$AA?$CJ?$AA?$AN?$AA?6?$AA?$AA@ 10001860     backlight_common_topaz_v1:backlight.obj
 0001:00000898       ??_C@_17JLFEDMMI@?$AA?$DP?$AA?$DP?$AA?$DP?$AA?$AA@ 10001898     backlight_common_topaz_v1:backlight.obj
 0001:000008a0       ??_C@_1BA@LEPJIIOK@?$AAU?$AAn?$AAk?$AAn?$AAo?$AAw?$AAn?$AA?$AA@ 100018a0     backlight_common_topaz_v1:backlight.obj
 0001:000008b0       ??_C@_1O@LKOFKKHD@?$AAB?$AAa?$AAc?$AAk?$AAu?$AAp?$AA?$AA@ 100018b0     backlight_common_topaz_v1:backlight.obj
 0001:000008c0       ??_C@_1BA@DKNJBOGI@?$AAO?$AAf?$AAf?$AAl?$AAi?$AAn?$AAe?$AA?$AA@ 100018c0     backlight_common_topaz_v1:backlight.obj
 0001:000008d0       ??_C@_15DJIHAEG@?$AAA?$AAC?$AA?$AA@ 100018d0     backlight_common_topaz_v1:backlight.obj
 0001:000008d8       ??_C@_1EI@NJMJAJD@?$AAP?$AAM?$AAA?$AAP?$AAI?$AA?$CB?$AAC?$AAe?$AAS?$AAe?$AAt?$AAT?$AAh?$AAr?$AAe?$AAa?$AAd?$AAP?$AAr?$AAi?$AAo?$AAr?$AAi?$AAt?$AAy?$AA?5?$AAE?$AAR?$AAR?$AAO?$AAR?$AA?3@ 100018d8     backlight_common_topaz_v1:backlight.obj
 0001:00000920       ??_C@_1EA@EEDKECB@?$AA?$CF?$AAs?$AA?3?$AA?5?$AAU?$AAn?$AAs?$AAu?$AAp?$AAp?$AAo?$AAr?$AAt?$AAe?$AAd?$AA?5?$AAI?$AAO?$AAC?$AAT?$AAL?$AA?5?$AAc?$AAo?$AAd?$AAe?$AA?5?$AA?$CF?$AAu?$AA?$AN?$AA?6?$AA?$AA@ 10001920     backlight_common_topaz_v1:backlight.obj
 0001:00000960       ??_C@_1DE@OLFDBLOE@?$AA?$CF?$AAs?$AA?3?$AA?5?$AAB?$AAK?$AAL?$AA_?$AAI?$AAO?$AAC?$AAT?$AAL?$AA_?$AAP?$AAO?$AAW?$AAE?$AAR?$AA_?$AAG?$AAE?$AAT?$AA?$AN?$AA?6?$AA?$AA@ 10001960     backlight_common_topaz_v1:backlight.obj
 0001:00000994       ??_C@_1BK@HEFCAJFH@?$AAC?$AAu?$AAr?$AAD?$AAx?$AA?5?$AA?$DN?$AA?5?$AA?$CF?$AAd?$AA?$AN?$AA?6?$AA?$AA@ 10001994     backlight_common_topaz_v1:backlight.obj
 0001:000009b0       ??_C@_1CA@JGOJPID@?$AAB?$AAa?$AAc?$AAk?$AAL?$AAi?$AAg?$AAh?$AAt?$AA?5?$AAO?$AAf?$AAf?$AA?$AN?$AA?6?$AA?$AA@ 100019b0     backlight_common_topaz_v1:backlight.obj
 0001:000009d0       ??_C@_1BO@PBBLIAOB@?$AAB?$AAa?$AAc?$AAk?$AAL?$AAi?$AAg?$AAh?$AAt?$AA?5?$AAO?$AAN?$AA?$AN?$AA?6?$AA?$AA@ 100019d0     backlight_common_topaz_v1:backlight.obj
 0001:000009f0       ??_C@_1DE@OEENMNGH@?$AA?$CF?$AAs?$AA?3?$AA?5?$AAB?$AAK?$AAL?$AA_?$AAI?$AAO?$AAC?$AAT?$AAL?$AA_?$AAP?$AAO?$AAW?$AAE?$AAR?$AA_?$AAS?$AAE?$AAT?$AA?$AN?$AA?6?$AA?$AA@ 100019f0     backlight_common_topaz_v1:backlight.obj
 0001:00000a24       ??_C@_1DM@DAMEDGF@?$AA?$CF?$AAs?$AA?3?$AA?5?$AAI?$AAO?$AAC?$AAT?$AAL?$AA_?$AAP?$AAO?$AAW?$AAE?$AAR?$AA_?$AAQ?$AAU?$AAE?$AAR?$AAY?$AA?5?$AA?$CF?$AAu?$AA?5?$AA?$CF?$AAs?$AA?$AN?$AA?6?$AA?$AA@ 10001a24     backlight_common_topaz_v1:backlight.obj
 0001:00000a60       ??_C@_1O@KPGHAGDD@?$AAf?$AAa?$AAi?$AAl?$AAe?$AAd?$AA?$AA@ 10001a60     backlight_common_topaz_v1:backlight.obj
 0001:00000a70       ??_C@_1BE@GCAFJAHI@?$AAs?$AAu?$AAc?$AAc?$AAe?$AAe?$AAd?$AAe?$AAd?$AA?$AA@ 10001a70     backlight_common_topaz_v1:backlight.obj
 0001:00000a84       ??_C@_1BK@NIBAJMFP@?$AAN?$AAe?$AAw?$AAD?$AAx?$AA?5?$AA?$DN?$AA?5?$AA?$CF?$AAd?$AA?$AN?$AA?6?$AA?$AA@ 10001a84     backlight_common_topaz_v1:backlight.obj
 0001:00000aa0       ??_C@_1DI@OLAMLPEG@?$AA?$CF?$AAs?$AA?3?$AA?5?$AAB?$AAK?$AAL?$AA_?$AAI?$AAO?$AAC?$AAT?$AAL?$AA_?$AAP?$AAO?$AAW?$AAE?$AAR?$AA_?$AAQ?$AAU?$AAE?$AAR?$AAY?$AA?$AN?$AA?6?$AA?$AA@ 10001aa0     backlight_common_topaz_v1:backlight.obj
 0001:00000ad8       ??_C@_1EG@JLFEBGKJ@?$AA?$CF?$AAs?$AA?3?$AA?5?$AAB?$AAK?$AAL?$AA_?$AAI?$AAO?$AAC?$AAT?$AAL?$AA_?$AAP?$AAO?$AAW?$AAE?$AAR?$AA_?$AAC?$AAA?$AAP?$AAA?$AAB?$AAI?$AAL?$AAI?$AAT?$AAI?$AAE?$AAS@ 10001ad8     backlight_common_topaz_v1:backlight.obj
 0001:00000b20       ??_C@_1JA@JJAJNBB@?$AA?$CF?$AAs?$AA?3?$AA?5?$AAI?$AAO?$AAC?$AAT?$AAL?$AA?3?$AA0?$AAx?$AA?$CF?$AAx?$AA?0?$AA?5?$AAI?$AAn?$AAB?$AAu?$AAf?$AA?3?$AA0?$AAx?$AA?$CF?$AAx?$AA?0?$AA?5?$AAI?$AAn?$AAB?$AAu@ 10001b20     backlight_common_topaz_v1:backlight.obj
 0001:00000bb0       ??_C@_1DO@BFEBJAFP@?$AAD?$AAl?$AAl?$AAE?$AAn?$AAt?$AAr?$AAy?$AA?3?$AA?5?$AAD?$AAL?$AAL?$AA_?$AAP?$AAR?$AAO?$AAC?$AAE?$AAS?$AAS?$AA_?$AAD?$AAE?$AAT?$AAA?$AAC?$AAH?$AA?$AN?$AA?6?$AA?$AA@ 10001bb0     backlight_common_topaz_v1:backlight.obj
 0001:00000bf0       ??_C@_1DO@LJPEFOLH@?$AAD?$AAl?$AAl?$AAE?$AAn?$AAt?$AAr?$AAy?$AA?3?$AA?5?$AAD?$AAL?$AAL?$AA_?$AAP?$AAR?$AAO?$AAC?$AAE?$AAS?$AAS?$AA_?$AAA?$AAT?$AAT?$AAA?$AAC?$AAH?$AA?$AN?$AA?6?$AA?$AA@ 10001bf0     backlight_common_topaz_v1:backlight.obj
 0001:00000c30       ??_C@_1BI@IJHODHIK@?$AA?9?$AAB?$AAK?$AAL?$AA_?$AAO?$AAp?$AAe?$AAn?$AA?$AN?$AA?6?$AA?$AA@ 10001c30     backlight_common_topaz_v1:backlight.obj
 0001:00000c48       ??_C@_1IA@IKFMNHKP@?$AA?$CL?$AAB?$AAK?$AAL?$AA_?$AAO?$AAp?$AAe?$AAn?$AA?3?$AA?5?$AAd?$AAw?$AAD?$AAa?$AAt?$AAa?$AA?5?$AA?$DN?$AA?5?$AA0?$AAx?$AA?$CF?$AAx?$AA?0?$AA?5?$AAd?$AAw?$AAA?$AAc?$AAc?$AAe@ 10001c48     backlight_common_topaz_v1:backlight.obj
 0001:00000cc8       ??_C@_1DI@NIDLHEL@?$AA?9?$AAB?$AAK?$AAL?$AA_?$AAC?$AAl?$AAo?$AAs?$AAe?$AA?3?$AA?5?$AAH?$AAa?$AAn?$AAd?$AAl?$AAe?$AA?5?$AA?$DN?$AA?5?$AA0?$AAx?$AA?$CF?$AAx?$AA?$AN?$AA?6?$AA?$AA@ 10001cc8     backlight_common_topaz_v1:backlight.obj
 0001:00000d00       ??_C@_1DI@EAPNNPLJ@?$AA?$CL?$AAB?$AAK?$AAL?$AA_?$AAC?$AAl?$AAo?$AAs?$AAe?$AA?3?$AA?5?$AAH?$AAa?$AAn?$AAd?$AAl?$AAe?$AA?5?$AA?$DN?$AA?5?$AA0?$AAx?$AA?$CF?$AAx?$AA?$AN?$AA?6?$AA?$AA@ 10001d00     backlight_common_topaz_v1:backlight.obj
 0001:00000d38       ??_C@_1CE@FEEMODNL@?$AAB?$AAK?$AAL?$AA_?$AAP?$AAO?$AAW?$AAE?$AAR?$AAD?$AAO?$AAW?$AAN?$AA?$CB?$AA?$CB?$AA?$AN?$AA?6?$AA?$AA@ 10001d38     backlight_common_topaz_v1:backlight.obj
 0001:00000d5c       ??_C@_1CA@PJACAJOB@?$AAB?$AAK?$AAL?$AA_?$AAP?$AAO?$AAW?$AAE?$AAR?$AAU?$AAP?$AA?$CB?$AA?$CB?$AA?$AN?$AA?6?$AA?$AA@ 10001d5c     backlight_common_topaz_v1:backlight.obj
 0001:00000d80       ??_C@_1HK@CGHPKHCD@?$AAB?$AAK?$AAL?$AA_?$AAR?$AAe?$AAa?$AAd?$AA?3?$AA?5?$AAH?$AAa?$AAn?$AAd?$AAl?$AAe?$AA?5?$AA?$DN?$AA?5?$AA0?$AAx?$AA?$CF?$AAx?$AA?0?$AA?5?$AAp?$AAB?$AAu?$AAf?$AAf?$AAe?$AAr@ 10001d80     backlight_common_topaz_v1:backlight.obj
 0001:00000e00       ??_C@_1HM@BGGEBIOG@?$AAB?$AAK?$AAL?$AA_?$AAW?$AAr?$AAi?$AAt?$AAe?$AA?3?$AA?5?$AAH?$AAa?$AAn?$AAd?$AAl?$AAe?$AA?5?$AA?$DN?$AA?5?$AA0?$AAx?$AA?$CF?$AAx?$AA?0?$AA?5?$AAp?$AAB?$AAu?$AAf?$AAf?$AAe@ 10001e00     backlight_common_topaz_v1:backlight.obj
 0001:00000e80       ??_C@_1IC@MJNFNLOK@?$AAB?$AAK?$AAL?$AA_?$AAS?$AAe?$AAe?$AAk?$AA?3?$AA?5?$AAH?$AAa?$AAn?$AAd?$AAl?$AAe?$AA?5?$AA?$DN?$AA?5?$AA0?$AAx?$AA?$CF?$AAx?$AA?0?$AA?5?$AAl?$AAD?$AAi?$AAs?$AAt?$AAa?$AAn@ 10001e80     backlight_common_topaz_v1:backlight.obj
 0001:00000f08       ??_C@_1FC@IPPMCHJD@?$AAG?$AAe?$AAt?$AA?5?$AAB?$AAa?$AAc?$AAk?$AAL?$AAi?$AAg?$AAh?$AAt?$AA?5?$AAA?$AAC?$AA?5?$AAl?$AAe?$AAv?$AAe?$AAl?$AA?5?$AAr?$AAe?$AAg?$AAi?$AAs?$AAt?$AAr?$AAy?$AA?5@ 10001f08     backlight_common_topaz_v1:backlight.obj
 0001:00000f5c       ??_C@_1CC@OPDEBLKM@?$AAA?$AAC?$AAB?$AAa?$AAc?$AAk?$AAl?$AAi?$AAg?$AAh?$AAt?$AAL?$AAe?$AAv?$AAe?$AAl?$AA?$AA@ 10001f5c     backlight_common_topaz_v1:backlight.obj
 0001:00000f80       ??_C@_1FG@CHNDEHPB@?$AAG?$AAe?$AAt?$AA?5?$AAB?$AAa?$AAc?$AAk?$AAL?$AAi?$AAg?$AAh?$AAt?$AA?5?$AAB?$AAa?$AAt?$AAt?$AA?5?$AAl?$AAe?$AAv?$AAe?$AAl?$AA?5?$AAr?$AAe?$AAg?$AAi?$AAs?$AAt?$AAr@ 10001f80     backlight_common_topaz_v1:backlight.obj
 0001:00000fd8       ??_C@_1CG@LFMPNLPM@?$AAB?$AAa?$AAt?$AAt?$AAB?$AAa?$AAc?$AAk?$AAl?$AAi?$AAg?$AAh?$AAt?$AAL?$AAe?$AAv?$AAe?$AAl?$AA?$AA@ 10001fd8     backlight_common_topaz_v1:backlight.obj
 0001:00001000       ??_C@_1EC@LOOLOEBJ@?$AAO?$AAp?$AAe?$AAn?$AA?5?$AAB?$AAa?$AAc?$AAk?$AAL?$AAi?$AAg?$AAh?$AAt?$AA?5?$AAr?$AAe?$AAg?$AAi?$AAs?$AAt?$AAr?$AAy?$AA?5?$AAf?$AAa?$AAi?$AAl?$AA?$CB?$AA?$CB?$AA?$AN?$AA?6@ 10002000     backlight_common_topaz_v1:backlight.obj
 0001:00001044       ??_C@_1CO@MGKPHPG@?$AAC?$AAo?$AAn?$AAt?$AAr?$AAo?$AAl?$AAP?$AAa?$AAn?$AAe?$AAl?$AA?2?$AAB?$AAa?$AAc?$AAk?$AAl?$AAi?$AAg?$AAh?$AAt?$AA?$AA@ 10002044     backlight_common_topaz_v1:backlight.obj
 0001:00001078       ??_C@_1FC@NOMMIFBG@?$AAG?$AAe?$AAt?$AA?5?$AAB?$AAa?$AAc?$AAk?$AAL?$AAi?$AAg?$AAh?$AAt?$AA?5?$AAU?$AAs?$AAe?$AA?5?$AAE?$AAx?$AAt?$AA?5?$AAc?$AAh?$AAe?$AAc?$AAk?$AA?5?$AAb?$AAo?$AAx?$AA?5@ 10002078     backlight_common_topaz_v1:backlight.obj
 0001:000010cc       ??_C@_1O@ILKHMLBG@?$AAU?$AAs?$AAe?$AAE?$AAx?$AAt?$AA?$AA@ 100020cc     backlight_common_topaz_v1:backlight.obj
 0001:000010e0       ??_C@_1FK@ONOEHIHK@?$AAG?$AAe?$AAt?$AA?5?$AAB?$AAa?$AAc?$AAk?$AAL?$AAi?$AAg?$AAh?$AAt?$AA?5?$AAU?$AAs?$AAe?$AA?5?$AAB?$AAa?$AAt?$AAt?$AAe?$AAr?$AAy?$AA?5?$AAC?$AAh?$AAe?$AAc?$AAk?$AA?5@ 100020e0     backlight_common_topaz_v1:backlight.obj
 0001:0000113c       ??_C@_1BG@LEIIKALA@?$AAU?$AAs?$AAe?$AAB?$AAa?$AAt?$AAt?$AAe?$AAr?$AAy?$AA?$AA@ 1000213c     backlight_common_topaz_v1:backlight.obj
 0001:00001158       ??_C@_1FG@LLGACKFI@?$AAG?$AAe?$AAt?$AA?5?$AAB?$AAa?$AAc?$AAk?$AAL?$AAi?$AAg?$AAh?$AAt?$AA?5?$AAA?$AAC?$AA?5?$AAt?$AAi?$AAm?$AAe?$AAo?$AAu?$AAt?$AA?5?$AAr?$AAe?$AAg?$AAi?$AAs?$AAt?$AAr@ 10002158     backlight_common_topaz_v1:backlight.obj
 0001:000011b0       ??_C@_1BE@PJBHBNNG@?$AAA?$AAC?$AAT?$AAi?$AAm?$AAe?$AAo?$AAu?$AAt?$AA?$AA@ 100021b0     backlight_common_topaz_v1:backlight.obj
 0001:000011c8       ??_C@_1FK@KIIJMNEH@?$AAG?$AAe?$AAt?$AA?5?$AAB?$AAa?$AAc?$AAk?$AAL?$AAi?$AAg?$AAh?$AAt?$AA?5?$AAB?$AAa?$AAt?$AAt?$AA?5?$AAt?$AAi?$AAm?$AAe?$AAo?$AAu?$AAt?$AA?5?$AAr?$AAe?$AAg?$AAi?$AAs@ 100021c8     backlight_common_topaz_v1:backlight.obj
 0001:00001224       ??_C@_1BO@PELGLPFE@?$AAB?$AAa?$AAt?$AAt?$AAe?$AAr?$AAy?$AAT?$AAi?$AAm?$AAe?$AAo?$AAu?$AAt?$AA?$AA@ 10002224     backlight_common_topaz_v1:backlight.obj
 0001:00001248       ??_C@_1EI@LDEDHMNI@?$AAB?$AAA?$AAC?$AAK?$AAL?$AAI?$AAG?$AAH?$AAT?$AA?5?$AAA?$AAC?$AA?5?$AAT?$AAI?$AAM?$AAE?$AAO?$AAU?$AAT?$AA?5?$AA?$DN?$AA?5?$AA?$CF?$AAd?$AA?5?$AAs?$AAe?$AAc?$AAo?$AAn?$AAd@ 10002248     backlight_common_topaz_v1:backlight.obj
 0001:00001290       ??_C@_1EM@IJMCAEMO@?$AAB?$AAA?$AAC?$AAK?$AAL?$AAI?$AAG?$AAH?$AAT?$AA?5?$AAB?$AAA?$AAT?$AAT?$AA?5?$AAT?$AAI?$AAM?$AAE?$AAO?$AAU?$AAT?$AA?5?$AA?$DN?$AA?5?$AA?$CF?$AAd?$AA?5?$AAs?$AAe?$AAc?$AAo@ 10002290     backlight_common_topaz_v1:backlight.obj
 0001:00001308       ?BSPBacklightInitialize@@YAXXZ 10002308 f   bspbacklight.obj
 0001:000015b0       ?BSPBacklightRelease@@YAXXZ 100025b0 f   bspbacklight.obj
 0001:000015dc       ?BSPBacklightSetIntensity@@YAXK@Z 100025dc f   bspbacklight.obj
 0001:0000170c       ?BSPBacklightEnable@@YAXXZ 1000270c f   bspbacklight.obj
 0001:00001710       BKL_Init                   10002710 f   backlight_common_topaz_v1:backlight.obj
 0001:00001eb0       BKL_Deinit                 10002eb0 f   backlight_common_topaz_v1:backlight.obj
 0001:0000209c       ?BKL_EventThread@@YAKPAX@Z 1000309c f   backlight_common_topaz_v1:backlight.obj
 0001:00002768       BKL_IOControl              10003768 f   backlight_common_topaz_v1:backlight.obj
 0001:00002e08       DllEntry                   10003e08 f   backlight_common_topaz_v1:backlight.obj
 0001:00002ec4       BKL_Open                   10003ec4 f   backlight_common_topaz_v1:backlight.obj
 0001:00002f58       BKL_Close                  10003f58 f   backlight_common_topaz_v1:backlight.obj
 0001:00002fe8       BKL_PowerDown              10003fe8 f   backlight_common_topaz_v1:backlight.obj
 0001:0000302c       BKL_PowerUp                1000402c f   backlight_common_topaz_v1:backlight.obj
 0001:00003070       BKL_Read                   10004070 f   backlight_common_topaz_v1:backlight.obj
 0001:000030d4       BKL_Write                  100040d4 f   backlight_common_topaz_v1:backlight.obj
 0001:00003138       BKL_Seek                   10004138 f   backlight_common_topaz_v1:backlight.obj
 0001:000037a8       SetEvent                   100047a8 f i backlight_common_topaz_v1:backlight.obj
 0001:000037dc       GetCurrentThread           100047dc f i backlight_common_topaz_v1:backlight.obj
 0001:000037f4       RegCloseKey                100047f4 f   coredll:COREDLL.dll
 0001:00003804       RegQueryValueExW           10004804 f   coredll:COREDLL.dll
 0001:00003814       RegOpenKeyExW              10004814 f   coredll:COREDLL.dll
 0001:00003824       CreateThread               10004824 f   coredll:COREDLL.dll
 0001:00003834       RequestPowerNotifications  10004834 f   coredll:COREDLL.dll
 0001:00003844       GetLastError               10004844 f   coredll:COREDLL.dll
 0001:00003854       CreateMsgQueue             10004854 f   coredll:COREDLL.dll
 0001:00003864       CreateEventW               10004864 f   coredll:COREDLL.dll
 0001:00003874       GetSystemPowerStatusEx     10004874 f   coredll:COREDLL.dll
 0001:00003884       InitializeCriticalSection  10004884 f   coredll:COREDLL.dll
 0001:00003894       NKDbgPrintfW               10004894 f   coredll:COREDLL.dll
 0001:000038a4       DeleteCriticalSection      100048a4 f   coredll:COREDLL.dll
 0001:000038b4       CloseMsgQueue              100048b4 f   coredll:COREDLL.dll
 0001:000038c4       StopPowerNotifications     100048c4 f   coredll:COREDLL.dll
 0001:000038d4       CloseHandle                100048d4 f   coredll:COREDLL.dll
 0001:000038e4       EventModify                100048e4 f   coredll:COREDLL.dll
 0001:000038f4       DevicePowerNotify          100048f4 f   coredll:COREDLL.dll
 0001:00003904       WaitForSingleObject        10004904 f   coredll:COREDLL.dll
 0001:00003914       GetSystemPowerStatusEx2    10004914 f   coredll:COREDLL.dll
 0001:00003924       ReadMsgQueue               10004924 f   coredll:COREDLL.dll
 0001:00003934       WaitForMultipleObjects     10004934 f   coredll:COREDLL.dll
 0001:00003944       CeSetThreadPriority        10004944 f   coredll:COREDLL.dll
 0001:00003954       SetLastError               10004954 f   coredll:COREDLL.dll
 0001:00003964       LeaveCriticalSection       10004964 f   coredll:COREDLL.dll
 0001:00003974       EnterCriticalSection       10004974 f   coredll:COREDLL.dll
 0001:00003984       RegisterDbgZones           10004984 f   coredll:COREDLL.dll
 0001:00003994       MmMapIoSpace               10004994 f   ceddk:CEDDK.dll
 0001:000039a4       MmUnmapIoSpace             100049a4 f   ceddk:CEDDK.dll
 0001:000039b4       DDKGpioWriteDataPin        100049b4 f   cspddk:CSPDDK.dll
 0001:000039c4       DDKGpioSetConfig           100049c4 f   cspddk:CSPDDK.dll
 0001:000039d4       DDKIomuxSetPadConfig       100049d4 f   cspddk:CSPDDK.dll
 0001:000039e4       DDKIomuxSetPinMux          100049e4 f   cspddk:CSPDDK.dll
 0001:000039f4       _DllEntryCRTStartup        100049f4 f   corelib0:pegdentry.obj
 0001:00003a60       __security_init_cookie     10004a60 f   corelib0:seccinit.obj
 0001:00003af8       __GSHandlerCheck           10004af8 f   corelib0:gshandler.obj
 0001:00003b3c       __GSHandlerCheckCommon     10004b3c f   corelib0:gshandler.obj
 0001:00003be0       __security_check_cookie    10004be0 f   corelib0:armsecgs.obj
 0001:00003bf0       __gsfailure                10004bf0     corelib0:armsecgs.obj
 0001:00003c34       exit                       10004c34 f   corelib0:cexit.obj
 0001:00003d58       _exit                      10004d58 f   corelib0:cexit.obj
 0001:00003d78       _cexit                     10004d78 f   corelib0:cexit.obj
 0001:00003d90       _c_exit                    10004d90 f   corelib0:cexit.obj
 0001:00003da8       _initterm                  10004da8 f   corelib0:crt0dat.obj
 0001:00003df4       _cinit                     10004df4 f   corelib0:crt0dat.obj
 0001:00003e24       __crt_ExitProcess          10004e24 f   corelib0:exitproc_proxy.obj
 0001:00003e50       GetCurrentProcess          10004e50 f i corelib0:exitproc_proxy.obj
 0001:00003e68       _onexit                    10004e68 f   corelib0:onexit.obj
 0001:00004044       atexit                     10005044 f   corelib0:onexit.obj
 0001:00004094       memcpy                     10005094 f   corelib1:COREDLL.dll
 0001:000040a4       __rt_udiv                  100050a4 f   corelib1:COREDLL.dll
 0001:000040b4       memset                     100050b4 f   corelib1:COREDLL.dll
 0001:000040c4       __security_gen_cookie2     100050c4 f   corelib1:COREDLL.dll
 0001:000040d4       __report_gsfailure         100050d4 f   corelib1:COREDLL.dll
 0001:000040e4       free                       100050e4 f   corelib1:COREDLL.dll
 0001:000040f4       realloc                    100050f4 f   corelib1:COREDLL.dll
 0001:00004104       malloc                     10005104 f   corelib1:COREDLL.dll
 0001:00004114       _msize                     10005114 f   corelib1:COREDLL.dll
 0001:00004124       TerminateProcess           10005124 f   coredll:COREDLL.dll
 0001:0000413c       __IMPORT_DESCRIPTOR_COREDLL 1000513c     coredll:COREDLL.dll
 0001:00004150       __IMPORT_DESCRIPTOR_CEDDK  10005150     ceddk:CEDDK.dll
 0001:00004164       __IMPORT_DESCRIPTOR_CSPDDK 10005164     cspddk:CSPDDK.dll
 0001:00004178       __NULL_IMPORT_DESCRIPTOR   10005178     coredll:COREDLL.dll
 0002:00000000       __imp_MmMapIoSpace         10006000     ceddk:CEDDK.dll
 0002:00000004       __imp_MmUnmapIoSpace       10006004     ceddk:CEDDK.dll
 0002:00000008       \177CEDDK_NULL_THUNK_DATA  10006008     ceddk:CEDDK.dll
 0002:0000000c       __imp_CreateThread         1000600c     coredll:COREDLL.dll
 0002:00000010       __imp_RequestPowerNotifications 10006010     coredll:COREDLL.dll
 0002:00000014       __imp_GetLastError         10006014     coredll:COREDLL.dll
 0002:00000018       __imp_CreateMsgQueue       10006018     coredll:COREDLL.dll
 0002:0000001c       __imp_CreateEventW         1000601c     coredll:COREDLL.dll
 0002:00000020       __imp_GetSystemPowerStatusEx 10006020     coredll:COREDLL.dll
 0002:00000024       __imp_InitializeCriticalSection 10006024     coredll:COREDLL.dll
 0002:00000028       __imp_NKDbgPrintfW         10006028     coredll:COREDLL.dll
 0002:0000002c       __imp_DeleteCriticalSection 1000602c     coredll:COREDLL.dll
 0002:00000030       __imp_CloseMsgQueue        10006030     coredll:COREDLL.dll
 0002:00000034       __imp_StopPowerNotifications 10006034     coredll:COREDLL.dll
 0002:00000038       __imp_RegOpenKeyExW        10006038     coredll:COREDLL.dll
 0002:0000003c       __imp_EventModify          1000603c     coredll:COREDLL.dll
 0002:00000040       __imp_DevicePowerNotify    10006040     coredll:COREDLL.dll
 0002:00000044       __imp_WaitForSingleObject  10006044     coredll:COREDLL.dll
 0002:00000048       __imp_GetSystemPowerStatusEx2 10006048     coredll:COREDLL.dll
 0002:0000004c       __imp_ReadMsgQueue         1000604c     coredll:COREDLL.dll
 0002:00000050       __imp_WaitForMultipleObjects 10006050     coredll:COREDLL.dll
 0002:00000054       __imp_CeSetThreadPriority  10006054     coredll:COREDLL.dll
 0002:00000058       __imp_SetLastError         10006058     coredll:COREDLL.dll
 0002:0000005c       __imp_LeaveCriticalSection 1000605c     coredll:COREDLL.dll
 0002:00000060       __imp_EnterCriticalSection 10006060     coredll:COREDLL.dll
 0002:00000064       __imp_RegisterDbgZones     10006064     coredll:COREDLL.dll
 0002:00000068       __imp_RegQueryValueExW     10006068     coredll:COREDLL.dll
 0002:0000006c       __imp_CloseHandle          1000606c     coredll:COREDLL.dll
 0002:00000070       __imp_RegCloseKey          10006070     coredll:COREDLL.dll
 0002:00000074       __imp__msize               10006074     corelib1:COREDLL.dll
 0002:00000078       __imp_malloc               10006078     corelib1:COREDLL.dll
 0002:0000007c       __imp_realloc              1000607c     corelib1:COREDLL.dll
 0002:00000080       __imp_free                 10006080     corelib1:COREDLL.dll
 0002:00000084       __imp___report_gsfailure   10006084     corelib1:COREDLL.dll
 0002:00000088       __imp_memcpy               10006088     corelib1:COREDLL.dll
 0002:0000008c       __imp___rt_udiv            1000608c     corelib1:COREDLL.dll
 0002:00000090       __imp_memset               10006090     corelib1:COREDLL.dll
 0002:00000094       __imp___security_gen_cookie2 10006094     corelib1:COREDLL.dll
 0002:00000098       __imp_TerminateProcess     10006098     coredll:COREDLL.dll
 0002:0000009c       \177COREDLL_NULL_THUNK_DATA 1000609c     coredll:COREDLL.dll
 0002:000000a0       __imp_DDKIomuxSetPadConfig 100060a0     cspddk:CSPDDK.dll
 0002:000000a4       __imp_DDKGpioSetConfig     100060a4     cspddk:CSPDDK.dll
 0002:000000a8       __imp_DDKGpioWriteDataPin  100060a8     cspddk:CSPDDK.dll
 0002:000000ac       __imp_DDKIomuxSetPinMux    100060ac     cspddk:CSPDDK.dll
 0002:000000b0       \177CSPDDK_NULL_THUNK_DATA 100060b0     cspddk:CSPDDK.dll
 0002:00000150       dpCurSettings              10006150     backlight_common_topaz_v1:backlight.obj
 0002:00000594       __security_cookie          10006594     corelib0:seccinit.obj
 0002:00000598       __security_cookie_complement 10006598     corelib0:seccinit.obj
 0002:0000062c       _exitflag                  1000662c     corelib0:cexit.obj
 0002:00000630       __onexitend                10006630     <common>
 0002:00000634       __onexitbegin              10006634     <common>

 entry point at        0001:000039f4

 Static symbols

 0001:00001494       ?GetModeFromRegistry@@YAPAULCD_MODE_INFO@@XZ 10002494 f   bspbacklight.obj
 0001:0000319c       ?GetBacklightLevelSettings@@YAXPAU_bklSettings@@@Z 1000419c f   backlight_common_topaz_v1:backlight.obj
 0001:00003388       ?GetBacklightTimeoutSettings@@YAXPAU_bklSettings@@@Z 10004388 f   backlight_common_topaz_v1:backlight.obj
 0001:00003700       ?CalculateTimeout@@YAKPAU_bklSettings@@@Z 10004700 f   backlight_common_topaz_v1:backlight.obj
 0001:00003c54       doexit                     10004c54 f   corelib0:cexit.obj
